:1000000020710010E9000000ED000000EF0000008A
:10001000F1000000F3000000F50000004289FFEF4E
:10002000000000000000000000000000F7000000D9
:10003000F900000000000000FB000000FD000000CF
:10004000FF000000293B0000FF000000FF0000004F
:10005000FF000000FF000000FF000000FF000000A4
:10006000FF000000FF000000FF000000FF00000094
:10007000FF000000FF000000FF000000FF00000084
:10008000FF000000FF000000FF000000FF00000074
:10009000FF000000FF000000FF000000FF00000064
:1000A000C13E0000FF000000FF000000FF00000054
:1000B000FF000000FF000000FF000000FF00000044
:1000C000FF000000FF000000FF000000DFF80CD080
:1000D00000F05AF800480047B14B000020710010B2
:1000E000D0F800D0D0F804F005480047FEE7FEE75E
:1000F000FEE7FEE7FEE7FEE7FEE7FEE7FEE7FEE7D8
:10010000CD00000010B50B4604461146184600F01D
:1001100027F8C4E9000110BD40EA01039B0703D0A2
:1001200009E008C9121F08C0042AFAD203E011F836
:10013000013B00F8013B521EF9D27047D2B201E0F8
:1001400000F8012B491EFBD270470022F6E710B5DC
:1001500013460A4604461946FFF7F0FF204610BD35
:1001600070B500242546002801DA01244042002908
:1001700001DA0125494200F019F8AC4200D04042B2
:10018000002C00D0494270BD064C074D06E0E068E7
:1001900040F0010394E8070098471034AC42F6D3CE
:1001A000FFF798FFE05500000056000030B50B4601
:1001B000014600202022012409E021FA02F59D4297
:1001C00005D303FA02F5491B04FA02F52844151E6B
:1001D000A2F10102F1DC30BD0B4880680B490A68CE
:1001E000801A4A6802EB4203C3EBC212B0EBC20FA3
:1001F00008D3074802224260C26B02F0FD02C263CC
:10020000002048607047000000000940DC0000103A
:10021000008000400B4900200867C86010224A6136
:100220008861C022CA6308498A680849C1E9002078
:1002300007490860074908607846074908600020B8
:10024000704700000080004000000940DC00001002
:1002500080000010840000108800001070B50F4C62
:1002600000250E46656000F04BF80D49000601D5EB
:10027000086870BD0B4B06EB46022068C2EBC61245
:100280009E68361AB6EBC20FFAD3074802224260C4
:10029000C26B02F0FD02C2636560E9E7DC0000109A
:1002A00080000010000009400080004070B500236D
:1002B000084D0AE0CE5C04885B1C86EA14269BB2DB
:1002C00035F8166086EA04240480521E92B2F1D2F8
:1002D00070BD0000F450000030B5054C0022855C74
:1002E000A35C521C1D4492B2CD54FF2AF7D930BDF5
:1002F000F44F00000020704700207047FFFFFFFF11
:100300002DE9F04341F288320023264C264D274E3A
:10031000904208D8642800D228B942F21072914263
:1003200001D8052907D28620206078462B603060EE
:100330008620BDE8F083DFF87890D9F80820DFF850
:100340007480D8F80070D21BD8F8047007EB470C03
:10035000CCEBC717B2EBC70F06D20520206078465A
:100360002B6030600520E4E7134A02275760D2F87B
:100370003CC00CF0FD0CC2F83CC040B1DFF83CC002
:10038000BCFBF0F04010D061576001205060D9F8FC
:100390000800C8E90001236078462B603060002027
:1003A000C7E70000800000108400001088000010E3
:1003B00000000940DC0000100080004080A812010D
:1003C0000948007828B1094900EBC00051F8200025
:1003D00000470749822008600649212008607846C6
:1003E0000549086082207047180100100855000078
:1003F0008000001084000010880000104FF480502E
:10040000704770479D1000002DE9FC410746002011
:1004100090460E46ADF8000004460EE0351B402D18
:1004200000D9402539192A460D4800F0ECFBAAB244
:100430000B496846FFF73AFF2C44B442EED3391912
:10044000424601A800F0DFFBBDF80000BDF8041033
:10045000884202D10120BDE8FC810020FBE70000BA
:10046000240100102DE9F0436B4C00208BB0A070EC
:10047000E070DFF8A8816A4F4FF4005620714FF406
:100480008079012519223146684600F0BCFB022222
:1004900016213046FFF7B8FF00287DD0DDF80E109A
:1004A000022206F11900FFF7AFFF002874D09DF873
:1004B0000010062929D2DFE801F029030329291CAD
:1004C000D8F87420DDF80A30521C93421DD2D8F8B7
:1004D0007400DDF80A30C01ADDF80E30401C984276
:1004E00013D3DDF80A00DDF80E30184490420CD822
:1004F0000CE0DDF80E00B0F5F42F00D9A570DDF8A2
:100500001200C0F30B40512800D0A570012903D080
:10051000022901D0052943D19DF808004A46400729
:1005200006F2194107D53F4800F06DFB3C493D48B4
:10053000FFF7D2FE02E03A4800F065FB0020099088
:10054000B888ADF824000999019889B2884200D092
:10055000A57000200990387B8DF824000999BDF81A
:100560000100C9B2884200D0A5709DF800000228A1
:1005700016D1386B0990DDF812000999884200D035
:10058000A5700020099097F834008DF8240009998F
:100590009DF80300C9B200E026E0884200D0A570B3
:1005A0009DF81800401EFE2800D2A570BDF801007D
:1005B000A0F57F41FF3901D0502802D19DF80300FA
:1005C00020B9684600F030FA00B9A570DDF80E00D9
:1005D0001B360644684600F027FA30B1E07880B157
:1005E000217988420DD012E0A5709DF8180010B94D
:1005F0002079401C2071E078401CC0B2E0700C28CB
:1006000001D3A57003E0A07800283FF43BAFA078A9
:100610000BB0BDE8F08300000C000010AC530000EC
:10062000240300102402001070B500F02BF81049CC
:10063000104D114E114C087050B1114900EBC00023
:1006400001EB800080688047000609D5206870BDF6
:10065000822020602120286078463060822070BD92
:1006600000202060286078463060002070BD0000C7
:100670001801001084000010880000108000001095
:100680000855000070B5002400BF00BF00BF00BFC8
:1006900000BF00BF00BF00BF00BF00BF00BF00BF62
:1006A00000BF00BF00BF00BF00BF00BF00BF00BF52
:1006B00000BF00BF00BF00BF00BF00BF00BF00BF42
:1006C00000BF00BF00BF00BF2D4E4FF48025F56373
:1006D0009F2001F087FD002001F084FD60F30704F6
:1006E000002001F07FFD60F30F24002001F07AFD6F
:1006F00060F31744B56300BF00BF00BF00BF00BF79
:1007000000BF00BF00BF00BF00BF00BF00BF00BFF1
:1007100000BF00BF00BF00BF00BF00BF00BF00BFE1
:1007200000BF00BF00BF00BF00BF00BF00BF00BFD1
:1007300000BF00BF00BF1349601A8C421AD00BDC07
:10074000A4F1C204B4F5A11414D0B4F5803F11D0C3
:10075000B4F5003F0BD10DE00B49401805D00B4913
:10076000401809D00A49C84201D1022400E00024FF
:10077000204670BD0324FBE7042402F0D7FDF7E711
:1007800000C00920C220180003FBD6FF00FFFEFFB7
:100790000001F8FF05498220086005492220086011
:1007A00078460449086082207047000080000010ED
:1007B0008400001088000010054982200860054967
:1007C00021200860784604490860822070470000B4
:1007D000800000108400001088000010054982206D
:1007E0000860054922200860784604490860822094
:1007F0007047000080000010840000108800001086
:100800002DE9F041144B154D154E1B78154C63B175
:100810009AB1154F03EBC30307EB83031B6998479A
:10082000000612D52068BDE8F081822020602120DA
:100830002860784630608220F5E786202060092015
:100840002860784630608620EDE700202060286030
:10085000784630600020E6E71801001084000010A0
:100860008800001080000010085500002DE9F041BC
:10087000144B154D154E1B78154C63B19AB1154F9D
:1008800003EBC30307EB83039B699847000612D56C
:100890002068BDE8F0818220206022202860784610
:1008A00030608220F5E786202060092028607846A5
:1008B00030608620EDE700202060286078463060B8
:1008C0000020E6E7180100108400001088000010E6
:1008D0008000001008550000F8B5184C184D194E4E
:1008E0002778194CDDF818C087B1BCF1000F15D07E
:1008F000CDF800C0DFF854C007EBC7070CEB870743
:10090000FF69B847000611D52068F8BD8220206035
:1009100022202860784630608220F8BD8620206042
:1009200009202860784630608620F8BD00202060CD
:100930002860784630600020F8BD000018010010E3
:10094000840000108800001080000010085500008E
:1009500070B50948022400F11F05816829B1007BA8
:10096000000607D4022003F07FFD2C7300F010FC7A
:10097000002070BD012070BD7D1F001010B50C4817
:100980000C4C8068A178884200D2A0700849A278F7
:100990004039822003F098FD032060700448A2785B
:1009A0001F308168891A81600021017310BD000029
:1009B0007D1F00108C00001001460007C00E0906C4
:1009C00000D5401C704700002DE9F041092000F0DF
:1009D0004BF8124800264FF47A770670C821384643
:1009E000FFF73CFC0E4CA06842F21075A168091A92
:1009F000A942FBD3C8213846FFF730FCA068A168A4
:100A0000091AA942FBD3C8213846FFF727FC05483D
:100A1000022186708171C670BDE8F0817C000010F3
:100A2000000009400C0000100021425C12B9491C72
:100A30001829FAD3182901D00020704701207047E7
:100A400001460020074ACB0703D053695B0200D55B
:100A50000120890704D55169890201D540F00200BF
:100A60007047000000C0092070B54F4B50B1596865
:100A7000042403250226052907D2DFE801F0072D0B
:100A80004C74910000205860986070BD042807D015
:100A9000052809D0012402287DD0012809D011E0C1
:100AA000032000F083F848E0BDE87040012000F02A
:100AB0007DB8032000F07AF80CE000BF00F086F863
:100AC0005C6070BD0E28FCD1032000F06FF802209E
:100AD00000F07CF80120F1E706280AD0032810D0A6
:100AE0000A2813D0092811D00D280FD00C28D7D0F0
:100AF00070BD032000F05AF8022000F067F85E6035
:100B000070BD032000F052F8012028E0032000F01F
:100B10004DF8022012E0062814D00A281BD009281C
:100B2000C7D00C28BCD00D28F0D00F28E8D1032066
:100B300000F03CF8022000F049F80120BDE87040C8
:100B400000F044B8986810F01F0F00F101009860A1
:100B5000D6D102201BE0032000F028F8022000F08C
:100B600035F85D6070BD072806D00A2898D00B289C
:100B700011D009289DD070BD022000F017F89868A8
:100B800010F03F0F00F101009860F4D10120BDE8A2
:100B9000704000F02BB8032000F008F802208DE729
:100BA0000628A6D08EE70000CC0000100649C20738
:100BB00002D04FF48002CA61800702D54FF40010C2
:100BC000C86100207047000000C009200649C20724
:100BD00002D04FF480028A61800702D54FF40010E2
:100BE000886100207047000000C0092010B504464D
:100BF000FFF726FF0346FFF7D9FF24EA0300FFF7BC
:100C0000E5FF002010BD10B50B4601460024184634
:100C1000FFF7F6FD204610BD0E4810B541780229B9
:100C200008D003290ED0042910D0052901D10021B4
:100C3000417010BD0848C07B2828FAD1BDE810409B
:100C400000F034B9BDE8104000F0A2BA822003F0F1
:100C50000BFCF7E78C0000107D1F001010B5144945
:100C6000022003F00BFA13498870487860B101281C
:100C70000ED0022003F0F8FB0D4902205F3108730B
:100C8000BDE8104000F084BABDE8104000F014B890
:100C900007484030C07B2A2805D02F2807D1BDE85F
:100CA000104000F035B9BDE8104000F075B910BD36
:100CB0003D1F00108C0000102DE9F0414A4D4B4CB7
:100CC0000021A878A4F1400202E0535C6354491C5F
:100CD00003468142F9D31F2B7CD1206844498842C6
:100CE00078D1424E60681F364FF001087060A068EE
:100CF000B060607B18B9A07B08B1102802D986F8D3
:100D00000C8063E0E07B1E28F9D011DC122833D080
:100D100006DC68B30328F2D1BDE8F04100F00EBA5A
:100D20001528ECD01A28EAD1BDE8F04100F07EB9D0
:100D300002272A282ED011DC232821D0252823D0D1
:100D40002828DCD100F08AF900282CD0207B00066E
:100D50001ED56F70BDE8F04100F0A8B82F2824D050
:100D60005528CCD05A28CAD1BDE8F04100F042B98C
:100D7000BDE8F04100F01EBABDE8F04100F03AB81D
:100D8000BDE8F04100F0B4B9BDE8F04100F08EB923
:100D9000022018E000F062F9002804D0207B000651
:100DA00010D485F80180BDE8F08100F057F90028E3
:100DB000F9D0207B000605D485F80180C5F828808D
:100DC000F1E707E0822003F04FFB3773BDE8F04105
:100DD00000F0DEB9822003F047FB022003F044FB61
:100DE00006206870DFE700008C0000107D1F0010F7
:100DF000555342431CB5FFF7ABFD00284ED02848A1
:100E00000A2206210388684604F060F8254800227B
:100E100080230270437082700121C1702021017112
:100E200043718271C27141220272542242724F2276
:100E300082724C22C272017341738173C173462264
:100E4000027450234374722383746923C3746E2322
:100E50000375742343758175C2756C220276612215
:100E60004276732282766822C27601774177817753
:100E7000C1779DF8011080F820109DF8021080F8CD
:100E800021109DF8031080F822109DF8041080F8BE
:100E90002310054924208870FFF770FD1CBD000059
:100EA000040400003D1F00108C00001070B5154DAB
:100EB0002C6B402C00D94024E86AE96902198A4267
:100EC00002D90C1A04216970214603F04BFF224617
:100ED0000D49822003F0F8FAE86A2044E862286BA2
:100EE000011B0A4829638268A2EB0402826005D0D4
:100EF0006978022901D00021017370BD0321697056
:100F0000F9E700008C000010240100109C1F001065
:100F10002DE9F0411D4CA178E06A4218E1698A424E
:100F200006D9081AA07005206070022003F09CFA10
:100F30000021A078164B174DE26A08E056186F5C46
:100F40009E5DBE4202D00021A16202E0491C8142A6
:100F5000F4D31118E162216B0A1A0E49226301F1E0
:100F60005F018B68A3EB0000886002D060780528E1
:100F700009D1A06A28B100200873BDE8F04100F053
:100F800007B90120F8E7BDE8F08100008C000010EF
:100F9000240100103D1F001010B5144CA178E06A28
:100FA0004218E1698A4206D9081AA07005206070CB
:100FB000022003F059FAA178E06A03F019FFA17842
:100FC000E06A0844E062206B421A094822638368A1
:100FD000A3EB0101816002D06178052905D10021D0
:100FE0000173BDE8104000F0D3B810BD8C000010B4
:100FF0009C1F001010B5FFF7ABFC002811D009486A
:1010000000210622017042708170C170017141712E
:101010008171C171044908208870BDE81040FFF754
:10102000ADBC10BD3D1F00108C00001010B5FFF7C7
:101030008FFC00280DD0074803210170002141706A
:101040008170C170044904208870BDE81040FFF72A
:1010500095BC10BD3D1F00108C000010114810B54C
:10106000D0F81110027D09BA21F0FF0111430E4A98
:101070004902D162C18A49BA490211638068884233
:101080000DD0822003F0F0F9022003F0EDF90549BC
:1010900002201F31087300F07BF8002010BD0120F2
:1010A00010BD00007D1F00108C00001010B5FFF770
:1010B0004FFC002816D00C4A0C48116A491E0B0E32
:1010C00003700B0C43700B0A8370C1700021017117
:1010D000417102238371C17108209070BDE81040F6
:1010E000FFF74CBC10BD00008C0000103D1F00102D
:1010F00010B5FFF72DFC00281AD00E4800210E4B2A
:101100000170417081700822C2701A6A140E047155
:10111000140C4471140A8471C27102220272417269
:101120008272C1720C209870BDE81040FFF726BC97
:1011300010BD00003D1F00108C00001010B5FFF71F
:1011400007FC00281FD010487021022201700021E6
:1011500041708270C1700171417181710A22C27146
:10116000017241728172C172302202730122427394
:101170008173C17301744174044912208870BDE801
:101180001040FFF7FBBB10BD3D1F00108C0000108E
:10119000064910B5044808600D22822003F094F936
:1011A00003490520487010BD555342539C1F001041
:1011B0008C000010094810B5816839B1007B000629
:1011C00001D5822000E0022003F04EF903490020FF
:1011D0001F310873BDE81040FFF7DABF7D1F001014
:1011E0002DE9FC5F8846044601A9414800F0C0FA99
:1011F000404D414E414FE0BB03208DF800002009D7
:101200008DF8010020018DF802004FF000098DF8E3
:10121000039000BF00BF00BF00BF00BF00BF00BF02
:1012200000BF00BF00BF00BF00BF00BF00BF00BFC6
:1012300000BF00BF00BF00BF00BF00BF00BF00BFB6
:1012400000BF00BF00BF00BF00BF00BF00BF00BFA6
:1012500000BFDFF8ACB04FF4802ACBF83CA00421EB
:10126000684600F0C9FF0024002000F0BBFFC0B2B8
:1012700000E005E08DF8040018F80410884208D05A
:101280008220286022203060784638608220BDE8C5
:10129000FC9F641CB4F5805FE6D3CBF838A000BF98
:1012A00000BF00BF00BF00BF00BF00BF00BF00BF46
:1012B00000BF00BF00BF00BF00BF00BF00BF00BF36
:1012C00000BF00BF00BF00BF00BF00BF00BF00BF26
:1012D00000BF00BF00BF00BF00BF00BF00BFC5F818
:1012E00000907846C6F8009038600020CFE70000F4
:1012F000E0930400800000108400001088000010BB
:1013000000C009202DE9F0474FF0000900BF00BFE1
:1013100000BF00BF00BF00BF00BF00BF00BF00BFD5
:1013200000BF00BF00BF00BF00BF00BF00BF00BFC5
:1013300000BF00BF00BF00BF00BF00BF00BF00BFB5
:1013400000BF00BF00BF00BF00BF00BF344E4FF45E
:101350008025F5639F2000F045FF002000F042FF4C
:1013600000F0FF08002000F03DFFC4B2002000F0B4
:1013700039FFC1B2B56300BF00BF00BF00BF00BFEF
:1013800000BF00BF00BF00BF00BF00BF00BF00BF65
:1013900000BF00BF00BF00BF00BF00BF00BF00BF55
:1013A00000BF00BF00BF00BF00BF00BF00BF00BF45
:1013B00000BF00BF00BF1B4D1B4E1C4FB8F1C20F3A
:1013C00001D1202C08D0822028602120306078466E
:1013D00038608220BDE8F0871548142912D01529FD
:1013E00013D0162915D0182916D0C0F80090002067
:1013F00000F0CEF8C5F800907846C6F80090386046
:101400000020E7E74FF4801101E04FF40011016084
:10141000EDE74FF48001FAE74FF08071F7E7000045
:1014200000C0092080000010840000108800001017
:10143000100100102DE9F04FDFF89480DFF894B030
:1014400089B00F0004464FF0000628D04FF48055B5
:1014500001462A466846FEF755FEDDE900A10591E2
:101460002A46214606A8FEF74DFEDDE906404FF06C
:101470000009BD1BC0F58051A94200D20D4620B124
:10148000544517D10599884214D1204601F026F819
:1014900000060FD5D8F8000009B0BDE8F08F86210E
:1014A000C8F800100921CBF8001079460A480160FD
:1014B0008620F1E72E44641C4846BE42D9D3C8F8C2
:1014C00000007946CBF80000034801600020E3E704
:1014D000800000108400001088000010014800689F
:1014E000704700001001001070B5044600BF00BF37
:1014F00000BF00BF00BF00BF00BF00BF00BF00BFF4
:1015000000BF00BF00BF00BF00BF00BF00BF00BFE3
:1015100000BF00BF00BF00BF00BF00BF00BF00BFD3
:1015200000BF00BF00BF00BF00BF00BF174E4FF499
:101530008025F563052000F055FE002000F052FEE6
:101540002070B56300BF00BF00BF00BF00BF00BF79
:1015500000BF00BF00BF00BF00BF00BF00BF00BF93
:1015600000BF00BF00BF00BF00BF00BF00BF00BF83
:1015700000BF00BF00BF00BF00BF00BF00BF00BF73
:1015800000BF00BF207800F0010070BD00C009203E
:101590002DE9F047744E80464FF080773068BC11DB
:1015A000724DB84249D100BF00BF00BF00BF00BFAD
:1015B00000BF00BF00BF00BF00BF00BF00BF00BF33
:1015C00000BF00BF00BF00BF00BF00BF00BF00BF23
:1015D00000BF00BF00BF00BF00BF00BF00BF00BF13
:1015E00000BF00BF00BFEC63152000F0FBFD002032
:1015F00000F0F8FD00F0FF09AC6300BF00BF00BFC2
:1016000000BF00BF00BF00BF00BF00BF00BF00BFE2
:1016100000BF00BF00BF00BF00BF00BF00BF00BFD2
:1016200000BF00BF00BF00BF00BF00BF00BF00BFC2
:1016300000BF00BF00BF00BF00BF00BF00BF00BFB2
:1016400000BF00BF00BF00BF00BF00BF00BF00BFA2
:1016500000BF00BF00BF00BF00BF00BF00BF00BF92
:1016600000BF00BF00BF00BF00BF00BF00BF00BF82
:1016700000BF00BF00BF00BF00BFEC63062000F04A
:10168000B1FDAC6300BF00BF00BF00BF00BF00BF23
:1016900000BF00BF00BF00BF00BF00BF00BF00BF52
:1016A00000BF00BF00BF00BF00BF00BF00BF00BF42
:1016B00000BF00BF00BF00BF00BF00BF00BF00BF32
:1016C00000BF00BF00BF00BF00BF00BF00BF00BF22
:1016D00000BF00BF00BF00BF00BF00BF00BF00BF12
:1016E00000BF00BF00BF00BF00BF00BF00BF00BF02
:1016F00000BF00BF00BF00BF00BF00BF00BF00BFF2
:1017000000BF00BFEC63012000F06CFD4FEA8800D1
:1017100000F068FD3068B84202D1484600F062FD32
:10172000AC6300BF00BF00BF00BF00BF00BF00BF71
:1017300000BF00BF00BF00BF00BF00BF00BF00BFB1
:1017400000BF00BF00BF00BF00BF00BF00BF00BFA1
:1017500000BF00BF00BF00BF00BF00BF00BF00BF91
:1017600000BFBDE8F08700001001001000C0092094
:101770002DE9F041084C0F460646A56806E0A06832
:10178000401BB04202D30120BDE8F0813846FFF78C
:10179000ABFE0028F3D1F7E7000009402DE9F04F38
:1017A00089B0DFF8F0805FEA020B4FF00006079186
:1017B0000FD04FF4805501462A466846FEF7A2FC3A
:1017C000DDE90047284603F059FA5FEA00090DD029
:1017D00017E086213048C8F80010092101607946D9
:1017E0002E480160862009B0BDE8F08F82212A488A
:1017F000C8F8001022210160794628480160822043
:10180000F1E7ABEB0605C7F580504FF0000AA842A0
:1018100000D20546B5F5805F04D02046494601F068
:101820003DF8D8B907982A46811907EB0900FEF759
:1018300073FC204600F052FE80B92046494600F075
:101840000DF958B920464946FFF7CAFC78B10AF1AC
:10185000010000F0FF0ABAF1030F05D3484603F078
:101860007BF9D8F80000BEE7BAF1000FE1D12E44B1
:101870000027641C5E45C4D3484603F06DF9064951
:101880000020C8F800000860794604480160002084
:10189000A9E70000800000108400001088000010FC
:1018A0002DE9FF4F8DB00D46DDF868900026684C9D
:1018B00007935FEA09013ED04FF4805701463A464C
:1018C0006846FEF71FFCDDE900B10C913A46691C41
:1018D0006846FEF717FCDDE90010CDE904013A4641
:1018E00068460F99FEF70EFCDDE90085A9EB0607B7
:1018F000C5F58050B84200D2074625B1D8457DD104
:101900000C9885427AD14FF4805003F0B7F95FEA22
:10191000000A1CD0D84550D10C9885424DD12A469A
:101920004FEA0830514600F031FF000619D5504605
:1019300003F012F97AE08620206046480921016010
:10194000784645490860862011B0BDE8F08F8220B6
:10195000206040482221016079463F480160822092
:10196000F2E70598804509D1049901EB0030C1F5F3
:101970008052514400F00AFF0006D8D4404600F0DF
:10198000ADFD0006D3D407983A46811905EB0A004D
:10199000FEF7C2FBEA194FEA0830514601F034FE67
:1019A0000006C4D40599884533D1049800EB013072
:1019B0000499C1F58052514427E0059988450AD120
:1019C000049800EB01300499C1F58052514600F0B3
:1019D000DDFE0006ABD4404600F080FD0006A6D434
:1019E00007983A4681190F98304401F00DFE000621
:1019F0009DD4059988450CD1049800E00DE000EBDA
:101A000001300499C1F58052514601F0FDFD0006F8
:101A10008DD4504603F0A0F80AE007983A468119A1
:101A20000F98304401F0F0FD000601D520688BE7E7
:101A30003E44002508F101084E45FFF457AF054923
:101A400000202060086078460349086000207BE79A
:101A50008000001084000010880000102DE9F34F72
:101A60000024484D484E494FC3B080464FF0820A8B
:101A70004FF0210BA14641A94548FFF779FE002808
:101A80006CD101F093F902208DF800004FEA181094
:101A90008DF8010004EB08108DF8020044988DF8D1
:101AA000039000EB04214FF4807201A8FEF734FB91
:101AB00000BF00BF00BF00BF00BF00BF00BF00BF2E
:101AC00000BF00BF00BF00BF00BF00BF00BF00BF1E
:101AD00000BF00BF00BF00BF00BF00BF00BF00BF0E
:101AE00000BF00BF00BF00BF00BF00BF00BF00BFFE
:101AF00028494FF48020C8634FF48271684600F093
:101B00007BFB24494FF48020886300BF00BF00BFE7
:101B100000BF00BF00BF00BF00BF00BF00BF00BFCD
:101B200000BF00BF00BF00BF00BF00BF00BF00BFBD
:101B300000BF00BF00BF00BF00BF00BF00BF00BFAD
:101B400000BF00BF00BF00BF00BF641CE4B2102C88
:101B500091D341A90E48FFF70BFE48B1C5F800A08C
:101B60007846C6F800B03860822045B0BDE8F08FF6
:101B700001F0D0F8C5F800907846C6F800903860BB
:101B80000020F2E7800000108400001088000010A0
:101B9000E093040000C0092030B5FF4800218162B5
:101BA000416821F440414160416C21F4404141F4DD
:101BB00000414164F9494FF400028A610A6822F445
:101BC00000020A60C26822F04072C260C26C22F059
:101BD000407242F00072C2644FF08052CA630B6AD6
:101BE00043F080530B62C36823F04063C360C36C4F
:101BF00023F0406343F00063C3645400CC630B6A7A
:101C000043F000530B62036923F00C030361036D7F
:101C100023F00C0343F0080303650223CB650B6C30
:101C200043F002030B64036923F030030361036D87
:101C300023F0300343F0200303650423CB650B6CD2
:101C400043F004030B64036923F0C0030361036DD5
:101C500023F0C00343F0800303650823CB650B6CBE
:101C600043F008030B64036923F440730361036DBD
:101C700023F4407343F4007303651023CB650D6CAC
:101C800045F010050D64456A25F040754562456EC6
:101C900025F0407545F000754566C1F89C20D1F8E7
:101CA000802042F08052C1F88020426A22F04062D7
:101CB0004262426E22F0406242F000624266C1F827
:101CC0009C40D1F8802042F00052C1F88020026987
:101CD00022F003020261026D42F00302026501225A
:101CE000CA650A6C42F001020A64026922F4405299
:101CF0000261026D22F44052026540228A650A6C3C
:101D000042F040020A64026822F4404242F4004277
:101D10000260026C22F4404242F400420264026813
:101D200022F4402242F400220260026C22F440229B
:101D300042F400220264426822F00C024260426CCB
:101D400022F00C0242645A03CA610A6822F400328B
:101D50000A60426822F030024260426C22F0300297
:101D600042649A03CA610C6824F480240C600469FC
:101D700024F440440461046D24F440440465802448
:101D8000CC650C6C24F080040C64C46844F04044BE
:101D9000C460C46C24F0404444F00044C46444680B
:101DA00024F4402444F480244460446C24F440240B
:101DB00044F400244464446824F4403444F48034FB
:101DC0004460446C24F4403444F400344464446873
:101DD00024F4404444F480444460446C24F440447B
:101DE00044F400444464C46844F44024C460C46CB3
:101DF00024F4402444F40024C464046824F030042F
:101E000044F010040460046C24F0300444F0200416
:101E10000464046824F0C00444F040040460046CCA
:101E200024F0C0040464046824F0404444F0804476
:101E30000460046C24F0404444F0004404644468AA
:101E400024F00304641C4460446C24F003044464E0
:101E5000046924F4403444F400340461046D24F42F
:101E6000403444F400340465046924F4402444F408
:101E700000240461046D24F440240465046824F003
:101E80000304A41C0460046C24F00304A41C046474
:101E9000046824F00C0444F008040460046C24F08A
:101EA0000C040464C46844F44034C460C46C24F476
:101EB000403444F40034C464C46844F44044C4600E
:101EC000C46C24F4404444F40044C464C46844F43E
:101ED0004074C460C46C24F4407444F40074C4645A
:101EE000C46824F03004C460C46C24F03004C464BA
:101EF0008A630A6A42F480220A62C26822F440526B
:101F0000C260C26C22F44052C2649A048A630C6AB2
:101F100044F480040C62446824F0407444F08074FB
:101F20004460446C24F040744464446824F44004E5
:101F300044F480044460446C24F440044464046821
:101F400024F440640460046C24F440640464202499
:101F5000CC610C6844F020040C60046824F44074E4
:101F60000460046C24F440740464CB610B6823F0B7
:101F700010030B60036923F440030361036D23F432
:101F800040030365C314CB650C6C24F400640C643B
:101F9000446824F4405403E000C0024000C009201B
:101FA0004460446C24F4405444F400544464CA61D2
:101FB0000A6842F480020A60426822F44062426089
:101FC000426C22F4406242F4006242649A028A61E6
:101FD0000A6842F400120A60426822F0406242F04D
:101FE00080624260426C22F0406242F000624264D1
:101FF000426822F0405242F080524260426C22F02D
:10200000405242F000524264C26822F0405242F014
:102010000052C260C26C42F04052C264C26922F4F3
:102020004022C261C26D22F4402242F40022C26505
:102030009A03CA670A6E42F000720A66026922F4C5
:1020400040120261026D22F4401202650215CA6557
:102050000C6C24F480640C64046924F04074046102
:10206000046D24F0407404658414CC650C6C24F475
:1020700080540C64C46824F4400444F48004C460B4
:10208000C46C24F4400444F40004C464C46824F020
:102090000304C460C46C24F00304A41CC46494014D
:1020A0008C630C6A44F480340C62046924F040644C
:1020B0000461046D24F0406444F000640465D400BD
:1020C000CC650C6C44F400540C64846824F44034F3
:1020D0008460846C24F4403444F4003484648415B3
:1020E0008C630C6A44F480740C62846824F4401499
:1020F0008460846C24F4401444F400148464CA633F
:102100000C6A44F480640C62846824F04054846057
:10211000846C24F0405444F0005484641401CC6373
:102120000C6A44F480440C62046824F440040460A3
:10213000046C44F440040464CB610B6823F4006332
:102140000B60036823F440130360036C43F44013F3
:102150000364CA61086820F48060086030BD000034
:1021600010B5FEF761FAFEF72BF904494FF400525F
:10217000C1E90020A0F5F420886010BD0000001027
:1021800006493022C1F80822C1F81002D1F8000235
:102190008006FBD5D1F814027047000000C0005043
:1021A0000948062101610721016000214161416266
:1021B00002214160C168C906FCD400E08168C168A1
:1021C0004907FBD4002070470080084000B50B464B
:1021D000024604E0002000F005F802F8010B5B1E47
:1021E000F8D200BD03498860C868C006FCD488687E
:1021F000704700000080084000B50B46024603E02F
:1022000012F8010BFFF7EEFF5B1EF9D200BD0000D4
:102210002DE9F84F6946384800F05AFC8227374CC0
:10222000374D384E4FF0220A002855D19DF8000056
:10223000800701D400F0BAFD00BF00BF00BF00BF9F
:1022400000BF00BF00BF00BF00BF00BF00BF00BF96
:1022500000BF00BF00BF00BF00BF00BF00BF00BF86
:1022600000BF00BF00BF00BF00BF00BF00BF00BF76
:1022700000BF00BF00BF00BFDFF88C904FF4802884
:10228000C9F83C806020FFF7ADFFC9F8388000BF77
:1022900000BF00BF00BF00BF00BF00BF00BF00BF46
:1022A00000BF00BF00BF00BF00BF00BF00BF00BF36
:1022B00000BF00BF00BF00BF00BF00BF00BF00BF26
:1022C00000BF00BF00BF00BF00BF00BF00BF694626
:1022D0000E4800F0FDFB38B127607846C5F800A035
:1022E00030608220BDE8F88F0020206028607846AA
:1022F00030600020F6E70000E0930400800000104A
:10230000840000108800001000C0092080C3C901AB
:102310002DE9F0474FF0000900BF00BF00BF00BF2C
:1023200000BF00BF00BF00BF00BF00BF00BF00BFB5
:1023300000BF00BF00BF00BF00BF00BF00BF00BFA5
:1023400000BF00BF00BF00BF00BF00BF00BF00BF95
:1023500000BF00BF00BF00BF314E4FF48025F563C2
:102360009F20FFF73FFF0020FFF73CFF00F0FF0832
:102370000020FFF737FFC4B20020FFF733FFC1B2E0
:10238000B56300BF00BF00BF00BF00BF00BF00BFFC
:1023900000BF00BF00BF00BF00BF00BF00BF00BF45
:1023A00000BF00BF00BF00BF00BF00BF00BF00BF35
:1023B00000BF00BF00BF00BF00BF00BF00BF00BF25
:1023C00000BF184D184E194FB8F1BF0F03D1252C7F
:1023D0000AD0262C08D08220286021203060784640
:1023E00038608220BDE8F0871148412912D04FF4AF
:1023F0008002422912D04A2910D0C0F80090002053
:1024000000F0D0FAC5F800907846C6F80090386021
:102410000020E7E74FF400110160F0E70260EEE70B
:1024200000C0092080000010840000108800001007
:10243000140100102DE9F04FDFF89480DFF894B01C
:1024400089B00F0004464FF0000628D04FF48055A5
:1024500001462A466846FDF755FEDDE900A10591D3
:102460002A46214606A8FDF74DFEDDE906404FF05D
:102470000009BD1BC0F58051A94200D20D4620B114
:10248000544517D10599884214D1204600F026F80A
:1024900000060FD5D8F8000009B0BDE8F08F8621FE
:1024A000C8F800100921CBF8001079460A480160ED
:1024B0008620F1E72E44641C4846BE42D9D3C8F8B2
:1024C00000007946CBF80000034801600020E3E7F4
:1024D0008000001084000010880000102DE9FC47E7
:1024E000044601A93B4800F0F3FA3B4D3B4EDFF8B0
:1024F000F09048B182202860222079463060822006
:10250000C9F80010BDE8FC879DF80400800701D4DD
:1025100000F04CFC20208DF8000020098DF801000F
:1025200020018DF8020000248DF8034000BF00BF99
:1025300000BF00BF00BF00BF00BF00BF00BF00BFA3
:1025400000BF00BF00BF00BF00BF00BF00BF00BF93
:1025500000BF00BF00BF00BF00BF00BF00BF00BF83
:1025600000BF00BF00BF00BF00BF00BFDFF8748026
:102570004FF48027C8F83C7004216846FFF73CFE02
:10258000C8F8387000BF00BF00BF00BF00BF00BF69
:1025900000BF00BF00BF00BF00BF00BF00BF00BF43
:1025A00000BF00BF00BF00BF00BF00BF00BF00BF33
:1025B00000BF00BF00BF00BF00BF00BF00BF00BF23
:1025C00000BF00BF2C60794634600020C9F80010BD
:1025D00098E70000E09304008000001084000010E1
:1025E0008800001000C009204FF4805070470000A0
:1025F00001480068704700001401001070B50446DF
:1026000000BF00BF00BF00BF00BF00BF00BF00BFD2
:1026100000BF00BF00BF00BF00BF00BF00BF00BFC2
:1026200000BF00BF00BF00BF00BF00BF00BF00BFB2
:1026300000BF00BF00BF00BF00BF00BF00BF00BFA2
:10264000174E4FF48025F5630520FFF7CBFD0020E2
:10265000FFF7C8FD2070B56300BF00BF00BF00BF1B
:1026600000BF00BF00BF00BF00BF00BF00BF00BF72
:1026700000BF00BF00BF00BF00BF00BF00BF00BF62
:1026800000BF00BF00BF00BF00BF00BF00BF00BF52
:1026900000BF00BF00BF00BF207800F0010070BD88
:1026A00000C0092070B5044600BF00BF00BF00BFD6
:1026B00000BF00BF00BF00BF00BF00BF00BF00BF22
:1026C00000BF00BF00BF00BF00BF00BF00BF00BF12
:1026D00000BF00BF00BF00BF00BF00BF00BF00BF02
:1026E00000BF00BF00BF00BF174E4FF48025F56349
:1026F0000520FFF777FD0020FFF774FD2070B5631C
:1027000000BF00BF00BF00BF00BF00BF00BF00BFD1
:1027100000BF00BF00BF00BF00BF00BF00BF00BFC1
:1027200000BF00BF00BF00BF00BF00BF00BF00BFB1
:1027300000BF00BF00BF00BF00BF00BF00BF00BFA1
:10274000207800F0010070BD00C0092070B50C4D6C
:102750000C4E0D4C2AB100F019F8000609D520687E
:1027600070BD862020600920286078463060862071
:1027700070BD00202060286078463060002070BD69
:102780008400001088000010800000102DE9FC5F1C
:102790003D4D3E4E3E4F5FEA020A8B4604464FF0E7
:1027A00000080DD001A93B4800F092F980B18220C9
:1027B000286021203060784638608220BDE8FC9F88
:1027C000C5F800807846C6F8008038600020F5E73C
:1027D00003208DF80000200C8DF80100200A8DF8F0
:1027E00002008DF8034000BF00BF00BF00BF00BF64
:1027F00000BF00BF00BF00BF00BF00BF00BF00BFE1
:1028000000BF00BF00BF00BF00BF00BF00BF00BFD0
:1028100000BF00BF00BF00BF00BF00BF00BF00BFC0
:1028200000BF00BF00BF1C4C4FF48029C4F83C908F
:1028300004216846FFF7E0FC51465846FFF7C6FC06
:10284000C4F8389000BF00BF00BF00BF00BF00BF8A
:1028500000BF00BF00BF00BF00BF00BF00BF00BF80
:1028600000BF00BF00BF00BF00BF00BF00BF00BF70
:1028700000BF00BF00BF00BF00BF00BF00BF00BF60
:1028800000BF00BF9CE70000800000108400001023
:1028900088000010E093040000C009202DE9FC47E7
:1028A0008A46044601A93A4800F012F9394D3A4ED9
:1028B000DFF8E89048B18220286022207946306015
:1028C0008220C9F80010BDE8FC8703208DF80000C5
:1028D00020098DF8010020018DF8020000248DF8F8
:1028E000034000BF00BF00BF00BF00BF00BF00BF6C
:1028F00000BF00BF00BF00BF00BF00BF00BF00BFE0
:1029000000BF00BF00BF00BF00BF00BF00BF00BFCF
:1029100000BF00BF00BF00BF00BF00BF00BF00BFBF
:1029200000BFDFF87C804FF48027C8F83C7004219A
:102930006846FFF761FCB9115046FFF747FCC8F83D
:10294000387000BF00BF00BF00BF00BF00BF00BFA6
:1029500000BF00BF00BF00BF00BF00BF00BF00BF7F
:1029600000BF00BF00BF00BF00BF00BF00BF00BF6F
:1029700000BF00BF00BF00BF00BF00BF00BF00BF5F
:1029800000BF2C60794634600020C9F800109AE737
:10299000E093040080000010840000108800001004
:1029A00000C0092070B5064600BF00BF00BF00BFD1
:1029B00000BF00BF00BF00BF00BF00BF00BF00BF1F
:1029C00000BF00BF00BF00BF00BF00BF00BF00BF0F
:1029D00000BF00BF00BF00BF00BF00BF00BF00BFFF
:1029E00000BF00BF00BF00BF384D4FF48024EC6330
:1029F0005020FFF7F7FBAC6300BF00BF00BF00BF74
:102A000000BF00BF00BF00BF00BF00BF00BF00BFCE
:102A100000BF00BF00BF00BF00BF00BF00BF00BFBE
:102A200000BF00BF00BF00BF00BF00BF00BF00BFAE
:102A300000BF00BF00BF00BF00BF00BF00BF00BF9E
:102A400000BF00BF00BF00BF00BF00BF00BF00BF8E
:102A500000BF00BF00BF00BF00BF00BF00BF00BF7E
:102A600000BF00BF00BF00BF00BF00BF00BF00BF6E
:102A700000BF00BF00BF00BFEC630120FFF7B2FB47
:102A8000B000FFF7AFFBAC6300BF00BF00BF00BFEB
:102A900000BF00BF00BF00BF00BF00BF00BF00BF3E
:102AA00000BF00BF00BF00BF00BF00BF00BF00BF2E
:102AB00000BF00BF00BF00BF00BF00BF00BF00BF1E
:102AC00000BF00BF00BF00BF70BD000000C00920F4
:102AD0002DE9F041084C0F460646A56806E0A068BF
:102AE000401BB04202D30120BDE8F0813846FFF719
:102AF00085FD0028F3D1F7E7000009402DE9F041FA
:102B0000084C0F460646A56806E0A068401BB04288
:102B100002D30120BDE8F0813846FFF7C3FD00284D
:102B2000F3D1F7E7000009402DE9F04F89B0DFF855
:102B3000D080DFF8D0B05FEA02094FF000060791BD
:102B40000FD04FF4805501462A466846FDF7DAFA61
:102B5000DDE90047284602F091F85FEA000A0DD04F
:102B600017E08621C8F800100921CBF8001079463B
:102B700025480160862009B0BDE8F08F8221C8F8A1
:102B800000102221CBF8001079461F4801608220F6
:102B9000F1E7A9EB0605C7F58050A84200D205462B
:102BA000B5F5805F04D020465146FFF777FE80B927
:102BB0002046FFF793FC60B907982A46811907EB76
:102BC0000A00FDF7A9FA2E442046514600F044FAC7
:102BD00028B1504601F0C0FFD8F80000CBE700272D
:102BE000641C4E45D5D3504601F0B6FF0020C8F80E
:102BF00000007946CBF80000034801600020BAE7E6
:102C00008000001084000010880000102DE9FE43B1
:102C10000F46044602A93A48FFF75AFF394D3A4E8B
:102C2000DFF8E88048B182202860222079463060B1
:102C30008220C8F80010BDE8FE839DF808008007D8
:102C400001D400F0B3F802208DF80000200C8DF8BC
:102C50000100200A8DF802008DF803408DF8047001
:102C600000BF00BF00BF00BF00BF00BF00BF00BF6C
:102C700000BF00BF00BF00BF00BF00BF00BF00BF5C
:102C800000BF00BF00BF00BF00BF00BF00BF00BF4C
:102C900000BF00BF00BF00BF00BF00BF00BF00BF3C
:102CA0001B4F4FF48024FC6305216846FFF7A4FA0C
:102CB000BC6300BF00BF00BF00BF00BF00BF00BFBC
:102CC00000BF00BF00BF00BF00BF00BF00BF00BF0C
:102CD00000BF00BF00BF00BF00BF00BF00BF00BFFC
:102CE00000BF00BF00BF00BF00BF00BF00BF00BFEC
:102CF00000BF0020286079463060C8F800109AE7CD
:102D0000E093040080000010840000108800001090
:102D100000C0092070B500BF00BF00BF00BF00BFEA
:102D200000BF00BF00BF00BF00BF00BF00BF00BFAB
:102D300000BF00BF00BF00BF00BF00BF00BF00BF9B
:102D400000BF00BF00BF00BF00BF00BF00BF00BF8B
:102D500000BF00BF00BF144C4FF48025E563042082
:102D6000FFF740FAA56300BF00BF00BF00BF00BF70
:102D700000BF00BF00BF00BF00BF00BF00BF00BF5B
:102D800000BF00BF00BF00BF00BF00BF00BF00BF4B
:102D900000BF00BF00BF00BF00BF00BF00BF00BF3B
:102DA00000BF00BF00BF70BD00C0092070B500BFEC
:102DB00000BF00BF00BF00BF00BF00BF00BF00BF1B
:102DC00000BF00BF00BF00BF00BF00BF00BF00BF0B
:102DD00000BF00BF00BF00BF00BF00BF00BF00BFFB
:102DE00000BF00BF00BF00BF00BF00BF00BF144C4A
:102DF0004FF48025E5630620FFF7F4F9A56300BFD3
:102E000000BF00BF00BF00BF00BF00BF00BF00BFCA
:102E100000BF00BF00BF00BF00BF00BF00BF00BFBA
:102E200000BF00BF00BF00BF00BF00BF00BF00BFAA
:102E300000BF00BF00BF00BF00BF00BF00BF70BD2C
:102E400000C009202DE9F05F114EDFF84890DFF84F
:102E500048A0150083460F464FF000080ED000240E
:102E60000AE0395D0BEB0400FFF7D0FE000602D547
:102E70003068BDE8F09F641CAC42F2D3C6F8008015
:102E80007946C9F800800020CAF80010F1E7000078
:102E90008000001084000010880000102DE9FF4F12
:102EA0008DB00D46DDF868900026684C07935FEA08
:102EB00009013ED04FF4805701463A466846FDF777
:102EC00021F9DDE900B10C913A46691C6846FDF72D
:102ED00019F9DDE90010CDE904013A4668460F9979
:102EE000FDF710F9DDE90085A9EB0607C5F580506F
:102EF000B84200D2074625B1D8457DD10C9885420D
:102F00007AD14FF4805001F0B9FE5FEA000A1CD07C
:102F1000D84550D10C9885424DD12A464FEA083009
:102F20005146FFF733FC000619D5504601F014FE58
:102F30007AE08620206046480921016078464549AC
:102F40000860862011B0BDE8F08F822020604048E4
:102F50002221016079463F4801608220F2E705980E
:102F6000804509D1049901EB0030C1F580525144EC
:102F7000FFF70CFC0006D8D44046FFF7AFFA000676
:102F8000D3D407983A46811905EB0A00FDF7C4F837
:102F9000EA194FEA08305146FFF754FF0006C4D43F
:102FA0000599884533D1049800EB01300499C1F5A7
:102FB0008052514427E0059988450AD1049800EBD6
:102FC00001300499C1F580525146FFF7DFFB00063E
:102FD000ABD44046FFF782FA0006A6D407983A46DB
:102FE00081190F983044FFF72DFF00069DD40599F5
:102FF00088450CD1049800E00DE000EB0130049905
:10300000C1F580525146FFF71DFF00068DD4504692
:1030100001F0A2FD0AE007983A4681190F98304462
:10302000FFF710FF000601D520688BE73E4400251E
:1030300008F101084E45FFF457AF05490020206014
:10304000086078460349086000207BE78000001094
:1030500084000010880000102DE9F34F83B004466F
:1030600001A97148FFF734FD704D714E714F4FF05B
:10307000820818B12120C5F800806CE09DF804009A
:10308000800701D4FFF792FEAD208DF800002009E3
:103090008DF8010020018DF802004FF0000B8DF833
:1030A00003B000BF00BF00BF00BF00BF00BF00BF34
:1030B00000BF00BF00BF00BF00BF00BF00BF00BF18
:1030C00000BF00BF00BF00BF00BF00BF00BF00BF08
:1030D00000BF00BF00BF00BF00BF00BF00BF00BFF8
:1030E00000BFDFF854914FF4802A5446C9F83CA041
:1030F00004216846FFF780F802210498FFF77CF866
:10310000C9F8384000BF00BF00BF00BF00BF00BF0C
:1031100000BF00BF00BF00BF00BF00BF00BF00BFB7
:1031200000BF00BF00BF00BF00BF00BF00BF00BFA7
:1031300000BF00BF00BF00BF00BF00BF00BF00BF97
:1031400000BF00BF022401A93748FFF7C1FC48B106
:103150002220C5F80080306078463860822005B0B3
:10316000BDE8F08F00BF00BF00BF00BF00BF00BFC1
:1031700000BF00BF00BF00BF00BF00BF00BF00BF57
:1031800000BF00BF00BF00BF00BF00BF00BF00BF47
:1031900000BF00BF00BF00BF00BF00BF00BF00BF37
:1031A00000BF00BFC9F83CA0AD20FFF71BF8049892
:1031B00002212044FFF720F8C9F838A000BF00BF63
:1031C00000BF00BF00BF00BF00BF00BF00BF00BF07
:1031D00000BF00BF00BF00BF00BF00BF00BF00BFF7
:1031E00000BF00BF00BF00BF00BF00BF00BF00BFE7
:1031F00000BF00BF00BF00BF00BF00BFA41CA4B23F
:10320000B4F5805F9FD301A90748FFF761FC002850
:103210007FF430AFFFF77EFDC5F800B07846C6F802
:1032200000B0386000209AE7E093040080000010AE
:10323000840000108800001000C009204FF4805066
:1032400070474FF4800070472DE9F04F89B0DFF8E8
:10325000D080DFF8D0B05FEA02094FF00006079196
:103260000FD04FF4805501462A466846FCF74AFFC6
:10327000DDE90047284601F001FD5FEA000A0DD0B4
:1032800017E08621C8F800100921CBF80010794614
:1032900025480160862009B0BDE8F08F8221C8F87A
:1032A00000102221CBF8001079461F4801608220CF
:1032B000F1E7A9EB0605C7F58050A84200D2054604
:1032C000B5F5805F04D020465146FFF7E7FA80B994
:1032D0002046FFF703F960B907982A46811907EBE2
:1032E0000A00FCF719FF2E442046514600F096FADA
:1032F00028B1504601F030FCD8F80000CBE7002799
:10330000641C4E45D5D3504601F026FC0020C8F879
:1033100000007946CBF80000034801600020BAE7BE
:103320008000001084000010880000102DE9FF4785
:1033300003A93B48FFF7E2FB3A4D3B4EDFF8EC9028
:1033400050B1822028602120794630608220C9F85F
:10335000001004B0BDE8F0879DF80C00800701D490
:10336000FFF724FD42208DF800000024CDF8014035
:10337000CDF80540ADF8094000BF00BF00BF00BF59
:1033800000BF00BF00BF00BF00BF00BF00BF00BF45
:1033900000BF00BF00BF00BF00BF00BF00BF00BF35
:1033A00000BF00BF00BF00BF00BF00BF00BF00BF25
:1033B00000BF00BF00BF00BFDFF874804FF480275C
:1033C000C8F83C700B216846FEF716FFC8F8387045
:1033D00000BF00BF00BF00BF00BF00BF00BF00BFF5
:1033E00000BF00BF00BF00BF00BF00BF00BF00BFE5
:1033F00000BF00BF00BF00BF00BF00BF00BF00BFD5
:1034000000BF00BF00BF00BF00BF00BF00BF00BFC4
:103410002C60794634600020C9F8001099E700005C
:10342000E093040080000010840000108800001069
:1034300000C009202DE9F34F85B0044603A96D486B
:10344000FFF75CFB6C4D6D4E6D4F4FF0820B18B16A
:103450002120C5F800B060E0FFF7A8FC42208DF8FD
:1034600000004FF0000ACDF801A0CDF805A0ADF89E
:1034700009A000BF00BF00BF00BF00BF00BF00BF6A
:1034800000BF00BF00BF00BF00BF00BF00BF00BF44
:1034900000BF00BF00BF00BF00BF00BF00BF00BF34
:1034A00000BF00BF00BF00BF00BF00BF00BF00BF24
:1034B00000BFDFF850914FF48028C9F83C800B2101
:1034C0006846FEF799FEC9F8388000BF00BF00BF0C
:1034D00000BF00BF00BF00BF00BF00BF00BF00BFF4
:1034E00000BF00BF00BF00BF00BF00BF00BF00BFE4
:1034F00000BF00BF00BF00BF00BF00BF00BF00BFD4
:1035000000BF00BF00BF00BF00BF03A93948FFF7DD
:10351000F5FA48B12220C5F800B03060784638602E
:10352000822007B0BDE8F08F9DF80C00800701D421
:10353000FFF73CFC02208DF80000200C8DF8010004
:10354000200A8DF8020006988DF803408DF80400DB
:1035500000BF00BF00BF00BF00BF00BF00BF00BF73
:1035600000BF00BF00BF00BF00BF00BF00BF00BF63
:1035700000BF00BF00BF00BF00BF00BF00BF00BF53
:1035800000BF00BF00BF00BF00BF00BF00BF00BF43
:103590004446C846C9F83C4005216846FEF72CFE63
:1035A000C8F8384000BF00BF00BF00BF00BF00BF69
:1035B00000BF00BF00BF00BF00BF00BF00BF00BF13
:1035C00000BF00BF00BF00BF00BF00BF00BF00BF03
:1035D00000BF00BF00BF00BF00BF00BF00BF00BFF3
:1035E00000BF00BFC5F800A07846C6F800A038604C
:1035F000002096E7E0930400800000108400001093
:103600008800001000C009202DE9F05F114EDFF89E
:103610004890DFF848A0150083460F464FF0000899
:103620000ED000240AE0395D0BEB0400FFF702FF27
:10363000000602D53068BDE8F09F641CAC42F2D3AE
:10364000C6F800807946C9F800800020CAF800104A
:10365000F1E70000800000108400001088000010D6
:103660002DE9FF4F8DB00D46DDF868900026684CBF
:1036700007935FEA09013ED04FF4805701463A466E
:103680006846FCF73FFDDDE900B10C913A46691C44
:103690006846FCF737FDDDE90010CDE904013A4644
:1036A00068460F99FCF72EFDDDE90085A9EB0607BA
:1036B000C5F58050B84200D2074625B1D8457DD126
:1036C0000C9885427AD14FF4805001F0D7FA5FEA26
:1036D000000A1CD0D84550D10C9885424DD12A46BD
:1036E0004FEA08305146FFF751F8000619D5504609
:1036F00001F032FA7AE08620206046480921016014
:10370000784645490860862011B0BDE8F08F8220D8
:10371000206040482221016079463F4801608220B4
:10372000F2E70598804509D1049901EB0030C1F515
:1037300080525144FFF72AF80006D8D44046FEF7DD
:10374000CDFE0006D3D407983A46811905EB0A004E
:10375000FCF7E2FCEA194FEA08305146FFF754FF44
:103760000006C4D40599884533D1049800EB013094
:103770000499C1F58052514427E0059988450AD142
:10378000049800EB01300499C1F580525146FEF7D0
:10379000FDFF0006ABD44046FEF7A0FE0006A6D40F
:1037A00007983A4681190F983044FFF72DFF00061D
:1037B0009DD4059988450CD1049800E00DE000EBFC
:1037C00001300499C1F580525146FFF71DFF0006F4
:1037D0008DD4504601F0C0F90AE007983A468119A5
:1037E0000F983044FFF710FF000601D520688BE7E3
:1037F0003E44002508F101084E45FFF457AF054946
:1038000000202060086078460349086000207BE7BC
:103810008000001084000010880000102DE9F34F94
:1038200000244A4D4A4E4B4FC3B080464FF0820AA7
:103830004FF0210BA14641A94748FFF75FF9002847
:1038400070D19DF80401800701D4FFF7AFFA022080
:103850008DF800004FEA18108DF8010004EB0810F5
:103860008DF8020044988DF8039000EB04214FF48A
:10387000807201A8FCF750FC00BF00BF00BF00BF72
:1038800000BF00BF00BF00BF00BF00BF00BF00BF40
:1038900000BF00BF00BF00BF00BF00BF00BF00BF30
:1038A00000BF00BF00BF00BF00BF00BF00BF00BF20
:1038B00000BF00BF00BF00BF28494FF48020C8638D
:1038C0004FF482716846FEF797FC24494FF480203C
:1038D000886300BF00BF00BF00BF00BF00BF00BFC4
:1038E00000BF00BF00BF00BF00BF00BF00BF00BFE0
:1038F00000BF00BF00BF00BF00BF00BF00BF00BFD0
:1039000000BF00BF00BF00BF00BF00BF00BF00BFBF
:1039100000BF641CE4B2102C8DD341A90E48FFF700
:10392000EDF848B1C5F800A07846C6F800B0386098
:10393000822045B0BDE8F08FFFF7ECF9C5F80090A4
:103940007846C6F8009038600020F2E7800000104A
:103950008400001088000010E093040000C00920DB
:10396000F8B51446074E0A460B19716800258B42BC
:1039700000D90A1B034600943068FCF7ADFF2846C7
:10398000F8BD00000000001070B5034608468D1811
:103990000549002449688D4200D9881A1946FCF768
:1039A00065FF204670BD000000000010064802219F
:1039B00041600021016741611122C260C1630121A0
:1039C0004160002070470000000009404E4810B5DB
:1039D0002021C0F8A01100BFD0F8A0114906FBD5E6
:1039E0000321C0F80411494AC0F8A8214FF48062AD
:1039F000C0F8AC210122C0F80C210B23C0F88430A0
:103A0000C0F88020AA22C0F88C205523C0F88C3042
:103A1000D0F888406401FBD5C0F88010C0F88C2035
:103A2000C0F88C300521C0F808113949C0F8C4101D
:103A30000021C0F8C811D0F888106FEA11618A0718
:103A40003449D0F80C2102F0030207D07AB3012ADE
:103A500044D0022A47D0032A4ED13AE02AB1012AA3
:103A600013D0022A24D0032A46D1D0F88820D0F8D7
:103A70000431C2F30742DBB2521C5B1C5A43D0F83C
:103A80008830254CC3F30E030EE0D0F88820D0F820
:103A90000431C2F30742DBB2521C5B1C5A43D0F81C
:103AA00088301E4CC3F30E035B1C634321E010E01F
:103AB000D0F88820D0F80431C2F30742DBB2521CA0
:103AC0005B1C5A43D0F888304FF47A44C3F30E039A
:103AD000EAE7D0F80421124BD2B209E0D0F8042171
:103AE000104BD2B204E0D0F804214FF4FA43D2B222
:103AF000521CB3FBF2F20A60016821F4704141F4F8
:103B00004051016010BD000000C00F4000101103C3
:103B1000DE97E8A7D800001000127A0000366E0188
:103B200000093D00001BB70010B54FF040210120F7
:103B30000860FCF751FB10BD00B5FCF73DFF0449E0
:103B40005DF804EB41EA0040891300F015BD000068
:103B50000005400010B502468078FCF72DFF0B49A8
:103B6000D1F84432012484402343C1F84432C1F8DF
:103B700048029088C1F84C02D1F80002C005FBD57C
:103B80004FF48070C1F8080210BD000000C0005062
:103B900010B500B101204FF4807444EA0041074899
:103BA00000F0EAFC06480321C0F84412D0F80012E5
:103BB000C905FBD5C0F8084210BD00000005D800BB
:103BC00000C0005010B5040001D0012000E000202A
:103BD0004FF4807141EA0041054800F0CDFC0549F1
:103BE0004FF000700CB1886710BDC86710BD0000B1
:103BF0000005FE0000C0092010B5084CA288402A2C
:103C000000D940228020216800F05EFC2168014438
:103C10002160A188081AA08010BD0000F8000010E3
:103C200010B5064C0020216800F028FA21680144F4
:103C30002160A188081AA08010BD0000F8000010C3
:103C40007047000000B5FCF7B7FE04495DF804EBCF
:103C500041EA0040024900F08FBC0000000540002E
:103C60000001200000B5FCF7A7FE04495DF804EB55
:103C700041EA0040891300F07FBC000000054000CD
:103C80002DE9F0414A4C0027A4F108062178A4F15F
:103C90001C05082864D2DFE800F0630465746363E0
:103CA000868400F0F1FB2078C009FFF7C9FFE088A7
:103CB000B0802078C0F34111F1BB61780C294BD260
:103CC000DFE801F006094A0B4A101B1E202632438A
:103CD00000F0B6F84EE0002000E0012000F05CFAB1
:103CE00050B306E010F01F0F36D1A07840F08000EE
:103CF0002870BDE8F04100F0CDBB00F065F839E078
:103D000000202AE010F01F0F26D129481B381AE0A6
:103D100010F01F0F20D100F087FA68B100F0BAFB55
:103D2000BDE8F041FCF76DBB00F01F00012813D186
:103D3000687808B1207900E00EE0A97888420BD2BB
:103D40001B490C39084430601DE000F01F000128B9
:103D500002D100F011FBC3E7802000F085FBB780A3
:103D6000BDE8F081080608D4B0880028F8D0FFF735
:103D700057FFB0880028EFD0F2E7BDE8F04100F02F
:103D80008FBB080603D5BDE8F041FFF735BF2878A3
:103D90000106E5D500F07F002870BDE8F04100F095
:103DA000E7B9802000E00020BDE8F041FFF7C4BE85
:103DB00000010010022803D0032803D1FCF72CBF18
:103DC000FCF74CBF70470000194810B5007810F0A0
:103DD0001F0F1748C07829D115490839012806D086
:103DE000134A0228937806D003281FD112E0114805
:103DF0000860122012E01048002204E004780CB1A0
:103E000044882044521C9342F8D1027872B1086071
:103E1000408803E009481844086000788A88824294
:103E200000D98880FFF7E8FE012010BD002010BDFA
:103E300000010010245400003654000057540000C4
:103E400070B51D481C4D0078A5F1080510F01F0441
:103E50000AD01948A5F11401184B4A780079012CB1
:103E600006D0022C26D109E01348183828601DE03E
:103E700002B3897888421DD2002015E000F08F043B
:103E8000200605D504F00F064FF48030B04001E065
:103E90000120A0400AB922070CD18A68024209D049
:103EA000C9680142E8D0012018802B60FFF7A4FE0A
:103EB000012070BD002070BD00010010E020001046
:103EC0002DE9F0412F4DD5F80032C5F8083218071A
:103ED00021D52D4800F042FB2C48FEF751F9C106D0
:103EE00005D500F001F9BDE8F04100F035B98107D2
:103EF00005D5BDE8F04100F0010000F079B80107F8
:103F000009D5400703D5BDE8F04100F0CFBABDE8C0
:103F1000F04100F02BB91E4E58074FF001071DD499
:103F2000BDE8F0815FF00004D5F8302207FA04F113
:103F30000A4210D06008C5F8381200BFD5F8001248
:103F40008906FBD5D5F81412E2070CD056F82010DC
:103F500009B103208847641C202CE5D3D5F8300232
:103F60000028DFD1DCE73CB9490705D5316819B134
:103F7000012088470124D7E756F820100029EAD00D
:103F80000220E7E700C000500005FE000002FE002E
:103F9000C8540000134800B5C16821F0405141F0F9
:103FA0000051C160C16C41F04051C1640E491A20FA
:103FB0000860091D0A6830EA0202FBD14FF0E021D7
:103FC0004FF08070C1F88002084B202283F8002453
:103FD000C1F8000100F088F800205DF804EB00F063
:103FE000C7B8000000C00240F4CF005018E000E065
:103FF000002802D1014901204870704708010010D3
:1040000070B5194C607820B30026184D012810D0E7
:1040100002280DD1A8686168401A1549884215D355
:104020001448406B400011D50120FFF7CBFD6670AE
:1040300070BDA8686168401A0F498842F8D3002013
:10404000FFF7C0FDA86860600220607026700C2039
:1040500005E020780028EBD1012020700D20BDE87C
:104060007040FCF701BD000008010010000009408D
:10407000A086010000C0092040420F0000F00F029E
:10408000012370B503EB8203154AC2F8283200BF42
:10409000D2F820321C05FBD5C3F309030024DD1C34
:1040A00005E000BFD2F8186241F8046B641CB4EB61
:1040B000950FF7D30021C2F8281241F24821C140E0
:1040C000C9070AD1FCF778FC4FF4A06141EA00402F
:1040D00000F044FA034800F041FA184670BD0000B1
:1040E00000C000500005F2000D480021C0F8481241
:1040F0004021C0F84C120122C0F84822C0F84C12EE
:10410000D0F80012C905FBD54FF0FF31C0F83812C6
:10411000C0F83412C0F808120C21C0F8041270471D
:1041200000C00050044800214FF00112818001704E
:104130004170C0E902217047E400001000B5FCF7AF
:104140003BFC04495DF804EB41EA0040891300F0B0
:1041500013BA00000005400010B5FFF7E3FF024965
:104160000020487010BD00000801001070470000DA
:1041700030B50749074D41EA00442146284600F082
:10418000FBF921462846BDE8304000F0F5B90000B3
:10419000000180000005D00070B502462148A0F162
:1041A0001C04017811F01F030146498804D0012B3B
:1041B00029D0022B27D111E0012924D132B10120CD
:1041C00000F080F9A08840F0020005E0002000F037
:1041D00079F9A08820F00200A08021E0007900F0A9
:1041E0008F00030605D500F00F034FF480359D4086
:1041F00001E00125854063782BB1030703D0A36854
:104200002B4200D009B1002070BD22B100F02CF982
:10421000E068284303E0FFF78FFCE068A843E06014
:10422000012070BD000100102DE9F84F504F002013
:104230000090B8784FF000094FF0010A4FF4803B2E
:10424000A7F11C0600286AD04A4C64E06078022876
:1042500004D0042840D005285BD140E06179B878CB
:10426000814237D170702079B070414900200C39FB
:1042700001F80090401C0428FAD301254FEA0608F3
:104280000AFA05F0D8F80810084202D02846FFF7CD
:10429000D9FCD8F808100BFA05F0084203D045F015
:1042A0008000FFF7CFFC6D1C102DE9D34FF00110FB
:1042B000C8E902090120FFF76BFCE0794006B8F875
:1042C000040002D540F0010001E020F00100A8F850
:1042D00004001EE060881DE0E078009019E000987E
:1042E000B8B9A07800F08F05280604D505F00F01B5
:1042F0000BFA01F001E00AFA05F0B168014320462B
:10430000B160FFF727FC2846FFF7ACFC2846FFF713
:1043100015FF207804442078002897D11FE086F804
:10432000019001245546D846B16805FA04F00842C8
:1043300002D02046FFF786FCB16808FA04F0084274
:1043400003D044F08000FFF77DFC641C102CEBD3FD
:104350004FF00110C6E902090020FFF719FCB878F8
:104360007178884202D10120BDE8F88F0020FBE778
:1043700000010010365400002DE9FC5F384D002785
:104380003E466878BB46B846002866D0BA46354CEB
:1043900005F11C095DE06078022804D0042808D0EB
:1043A000052854D119E06079697888424FD0608837
:1043B0004EE0A77899F80410E6784FF00008B9426B
:1043C00045D199F80200B04241D125484FF0010A89
:1043D000103010F807B0C65539E099F80410B9420A
:1043E00035D1A17801F08F010191090605D5019918
:1043F00001F00F024FF4803101E0019A0121914058
:10440000009199F80200B04213D1A8680843A8604F
:10441000E968009881432046E960FFF79BFB01981B
:10442000FFF720FC0198FFF789FE009948EA010890
:104430000DE05E450BD118EA010F08D1A86888434A
:10444000A860E8688843E8600198FFF7FBFB2078E4
:104450000444207800289ED15046BDE8FC9F00000F
:10446000E40000103654000000B5FCF7A5FA04493A
:104470005DF804EB41EA0040024900F07DB800001D
:10448000000540000001010001490020FFF7F6BDD2
:104490000001001000221146802000F015B8000035
:1044A00001490020FFF7EABDE02000100348012188
:1044B000417003498968416070470000080100109D
:1044C000000009407047000070B513460546134CC4
:1044D00000F00F00022202EB8000C4F82802C4F8AA
:1044E00024320020DA1C04E051F8046BC4F81C628A
:1044F000401CB0EB920FF7D30020C4F828022846E6
:10450000FCF75AFA4FF4A06141EA004000F026F8A7
:10451000034800F023F8184670BD000000C00050AA
:104520000005FA00EFF3108010F0010F72B64FF0A3
:1045300080404FF0000202704FF0AA0303724FF068
:104540005504047202614FF0FF0242604FF0030213
:1045500002700372047200D162B6FEE705491022B0
:10456000C1F80822C1F81002D1F80002C006FBD53C
:104570007047000000C00050094A1023C2F80832FA
:10458000C2F81002D2F80002C006FBD5C2F8083209
:10459000C2F81012D2F80002C006FBD57047000026
:1045A00000C0005002E008C8121F08C1002AFAD15A
:1045B00070477047002001E001C1121F002AFBD1A3
:1045C000704700000B4910B5486D00050CD40A4A2D
:1045D000906843F698239468241A9C42FBD3486D54
:1045E000000501D4012010BD0520FCF73DFA002094
:1045F00010BD000000C0092000000940F0B50546CC
:104600000020034602462B4C4FF4007700E05B1C71
:10461000EE5C46B102EB030CA4440CF5805C9CF804
:1046200000C8B445F3D0032B3FD302F5C05020445B
:10463000037F457FC67F03EB0523857F2D0405EBB4
:1046400006652B4451EA03052BD021B91A49496864
:1046500040318B4225D8194B00215518254405F5CA
:10466000805595F800585D54491C0C29F5D3817E7E
:10467000C27E01EB0221027D407D120402EB00604C
:104680000C18204600F030FB40F6F57502E000BF44
:1046900000F02AFBC11EA942FAD3A0F57061FF39D0
:1046A00001D00020F0BD2046F0BD2032BA42AFD389
:1046B000F0BD00003D0500108C000010A91F001087
:1046C00070B50D4CA6680420FCF7CEF90B4D02E046
:1046D000FFF778FF48B1A068801BA842F8D308E034
:1046E000FFF770FF08B1012070BDA068801BA842D1
:1046F000F6D3002070BD00000000094080841E0039
:104700008CB04FF00009CDF8289046208DF81400A9
:104710008DF8179038218DF81510DC4A3021CDF82E
:1047200024908DF816101168CA464FF6FF03194001
:10473000D74B41F4807119431160D649D648DA4D00
:10474000C1F800900068D549A0F56C50FF380860AA
:10475000D34900F5E0500860D249400A0860F820CB
:104760002870FF206870A870FBF754FDD04CCF4A2A
:10477000002094F9051052F821102B1803F58053EE
:104780000A5C401C83F800286028F6D34FF4E175DA
:10479000294640F24910FBF761FD294640F29F107F
:1047A000FBF75CFD4FF4005B5D46207808B1FFF736
:1047B00027FCA07938B101281BD0032873D02078BA
:1047C000002871D04BE10A20FCF74EF9FBF74AFEB6
:1047D00018B100BFFCF7F8F8E7E70120A0715D46CB
:1047E00084F803A00620FCF73FF90A20FCF73CF907
:1047F000DBE719222946AF48FCF705FAAD48007EF1
:10480000002875D0AB48007806285AD2DFE800F0BF
:10481000AC030B5A5A5D40F20440A649008804904C
:10482000496881424DD0A34F4FF00109787A0128A1
:1048300047D1D7F80A0018B99F488069C7F80A001D
:104840004FF4807800260720FCF70EF9D7F80E0009
:10485000B0422AD9801BFF2800D88046FF22511C75
:104860009648FBF76BFCA919424694481931FCF7AE
:10487000CAF9387A40070CD58E4990481931FBF7B0
:104880002BFDD7F80A008B4930444FF48072193160
:1048900005E0D7F80A004FF480723044874900F0F1
:1048A00079FB4644CFE7C0E0D2E0387801285BD1FD
:1048B0004FF0E0210006C1F88001D7F80A0000F0AF
:1048C0001DF951E04FF0010951E07A484FF001091C
:1048D000417A03294BD17049794A4FF000060B68A1
:1048E0001360027A520721D54FF48077804618E092
:1048F0005AE00720FCF7B8F8A9193A466F48193171
:10490000FCF781F96B496D481931FBF7E5FC62480A
:104910003A460068811967481930FFF721F806F513
:104920008076D8F80E00B042E3D81DE0804616E04D
:104930000720FCF799F8D7F80E00871B402F00D905
:104940004027A9193A465D481931FCF75CF95248ED
:104950003A46006881195948FFF702F83E44D8F8F2
:104960000E004746B042E3D85248007EE0B1514EB7
:10497000307AC00613D55249012204A8C1F800B00C
:1049800005F11801CDF810A0FEF7FEFF307820B138
:10499000C8214FF47A70FBF761FC307E20B1307A89
:1049A000800701D5FFF7BEFD42481B35D0F80E0049
:1049B00005444048FCF738F848B302204149A0714B
:1049C0005D4681F800A00B20FCF74EF8B9F1000F0E
:1049D0001DD03D484FF00009816842F21072836893
:1049E0005B1A9342FBD34FF42F714FF47A70FBF7AD
:1049F00035FC3648416DC90405D5406D400502D5EA
:104A000000200B9001E00B9808B9FFF78BFDE078D0
:104A1000401CC0B2E0700C2802D30120A070D9E67F
:104A2000A07800283FF4D8AED4E6274881680A98D9
:104A3000091A099800EB4002C2EBC010B1EBC00F9D
:104A4000FFF4CAAE00200A90099084F806A0ACE6F4
:104A500001202070FFF79EFA0120FFF7B3F81948F4
:104A600000780028F3D0002105A8FFF7C7FD002833
:104A7000EDD00320A071144884F803A05D4680683F
:104A80000A904FF47A7009908FE600000CED00E078
:104A90000000FA05C000001008000010B00000106F
:104AA000A8000010AC0000103D05001074000010BC
:104AB0000C000010240400103453000024010010E6
:104AC000000000107C0000100000094000C0092018
:104AD000084A34231360C2E9010107484FF47A7190
:104AE0000068B0FBF1F0D06002F11401104600F054
:104AF0005BB80000B81F0010D800001072B6034960
:104B0000034A01401160FBF7EBBA000080FFFF1F72
:104B100008ED00E010B572B606240E4951F82420C5
:104B2000824212D90B49783951F82410814207D1B9
:104B30002146084600F000F921460846FFF7C8FF65
:104B40002146084600F0F8F802E0641C1D2CE5D967
:104B500062B610BDAC53000010B5002821D0114B37
:104B60000022001F196803E0814203D80A46496801
:104B70000029F9D152B11368841A9C4204D100680B
:104B800018441060104602E0506000E0186039B12F
:104B900002680B1A934203D10B681A4402604968F9
:104BA000416010BD1C010010004A1047F11FFF1F9B
:104BB0002D4C0026FF202660A680A6716071FEF7AE
:104BC00005FFFCF7E9FFFEF7F1FEFBF795FB002080
:104BD000FBF74AFFFDF7E4FA244F786DC00402D5D5
:104BE000FFF7F0FC18B30420FBF73EFF786D204D73
:104BF000000514D4FFF764FDC8B1FFF761FDB0B143
:104C0000FFF75EFD98B10420FBF72EFFA868194955
:104C10007A6D120503D4AA68121A8A42F8D3A868DA
:104C200042F21071AA68121A8A42FBD36671FDF72C
:104C300097FAFBF717FC80B100F06CF968B102201D
:104C4000FBF712FF94F90500401C03D10A48806964
:104C5000FFF754FF0120607004E00220FBF704FF1F
:104C600066706671FFF74CFD0C00001000C0092053
:104C70000000094080841E0034530000F0B50B3062
:104C8000154D20F007010024144A0FE003688B4201
:104C90000BD38B4205D95E1A43184768C3E90067F6
:104CA00000E04368136002C004E0021D10680028A1
:104CB000ECD12046002802D1286808B10020F0BDC0
:104CC000064A07481060074A121A22F00702C0E994
:104CD000002401202860D7E7200100101C010010EB
:104CE0002421001020610010FFB50246002002EBD5
:104CF000420501464FF440566C4603AA6B1844F82F
:104D00002130B34202DD002004B0F0BD094F07EBB3
:104D10006307DB073F78575401D03B095354535C7A
:104D20008F0003F00F035354BB40491C1844032960
:104D3000E4DBE9E73D050010084A32231360C2E9CD
:104D4000010107484FF47A710068B0FBF1F0D060C0
:104D500002F114011046FFF727BF0000B81F001032
:104D6000D80000102DE9F0471D4A00234FF40077CA
:104D7000156A4FF4FF79C5F30724DFF868A04FF4F4
:104D8000E05CDFF86480194E25E0B84216D21328A3
:104D90000CD014280CD048450CD0A0F58072FF3AF6
:104DA0000AD03E2813D81AF8002011E0EAB20FE02A
:104DB00022460DE055220BE0AA2209E0604506D20A
:104DC00008EB0002A2F5805292F8002E00E00022CB
:104DD000F254401C5B1C8B42D7D3BDE8F087000027
:104DE0008C000010F45200003D050010240100105A
:104DF00070B50D462D494A6DD20402D5496D49055D
:104E000021D4B0F5007F1ED3294B2A4CB0F5E05FCA
:104E10001AD29968A269891A274A914204D39968DB
:104E2000A161002161606161244A0021A2F5D05393
:104E300007E044181C44565CA4F58054491C84F8CF
:104E4000006EA942F5D370BD616921B99968A1616D
:104E500099686161A0601A4949790029F3D199687C
:104E60006269891A174A91421BD2174A01211170AF
:104E70009968A16199686161A168401A6168884276
:104E800003D9616A884200D260600620FBF7ECFD1E
:104E900061682A46BDE87040084801F50051FEF7F8
:104EA0005FBDBDE870400C20FBF7DEBD00C00920EF
:104EB000000009408C000010A08601003D1F00107A
:104EC0000C00001020A107007C000010FFB50DA60B
:104ED0000446E1CE8DE8E100022902DA002004B0A8
:104EE000F0BD6018002100F8011D6946B3FBF2F522
:104EF00002FB1535B3FBF2F34D5D00F8015DA042F6
:104F0000F4D8ECE730313233343536373839414272
:104F10004344454610B546F204410023098846F251
:104F20003840A1F51942993A1AD002684FF4F4209A
:104F3000824200D902464FF4C0414C1E084622442A
:104F400001E010C823449042FBD94BB100204FF43C
:104F5000002208C991421844FBD308B1002010BDBB
:104F6000012010BD10B572B63324084B10C307C31F
:104F700007484FF47A710068B0FBF1F01860191D12
:104F80000248FFF711FE62B610BD0000B81F001006
:104F9000D80000102DE9F041144C236803B92060BB
:104FA0000020134D636803E00F5C1E18401CAF55D2
:104FB0009042F9D398184FF480766060B04212D1D5
:104FC0002068FFF7A7FD0A4D143D286800B1FEE7F1
:104FD000324607492068FFF7C5FF286800B1FEE7A1
:104FE0000020606020600020BDE8F081C400001057
:104FF000E01F001000050F0A1B1E141133363C3948
:10500000282D272263666C69787D777250555F5A28
:105010004B4E4441C3C6CCC9D8DDD7D2F0F5FFFA18
:10502000EBEEE4E1A0A5AFAABBBEB4B193969C9908
:10503000888D878283868C89989D9792B0B5BFBAF8
:10504000ABAEA4A1E0E5EFEAFBFEF4F1D3D6DCD9E8
:10505000C8CDC7C240454F4A5B5E545173767C79D8
:10506000686D676223262C29383D373210151F1AC8
:105070000B0E040103060C09181D171230353F3AB8
:105080002B2E242160656F6A7B7E747153565C59A8
:10509000484D4742C0C5CFCADBDED4D1F3F6FCF998
:1050A000E8EDE7E2A3A6ACA9B8BDB7B290959F9A88
:1050B0008B8E848180858F8A9B9E9491B3B6BCB978
:1050C000A8ADA7A2E3E6ECE9F8FDF7F2D0D5DFDA68
:1050D000CBCEC4C143464C49585D575270757F7A58
:1050E0006B6E646120252F2A3B3E343113161C1948
:1050F000080D070200002110422063308440A550B3
:10510000C660E770088129914AA16BB18CC1ADD10D
:10511000CEE1EFF13112100273325222B5529442B5
:10512000F772D662399318837BB35AA3BDD39CC35D
:10513000FFF3DEE36224433420040114E664C77401
:10514000A44485546AA54BB528850995EEE5CFF5AD
:10515000ACC58DD55336722611163006D776F66655
:105160009556B4465BB77AA719973887DFF7FEE7FD
:105170009DD7BCC7C448E5588668A7784008611821
:1051800002282338CCC9EDD98EE9AFF9488969994D
:105190000AA92BB9F55AD44AB77A966A711A500AF5
:1051A000333A122AFDDBDCCBBFFB9EEB799B588B9D
:1051B0003BBB1AABA66C877CE44CC55C222C033C41
:1051C000600C411CAEED8FFDECCDCDDD2AAD0BBDED
:1051D000688D499D977EB66ED55EF44E133E322E95
:1051E000511E700E9FFFBEEFDDDFFCCF1BBF3AAF3D
:1051F000599F788F8891A981CAB1EBA10CD12DC19B
:105200004EF16FE18010A100C230E3200450254030
:1052100046706760B9839893FBA3DAB33DC31CD390
:105220007FE35EF3B1029012F322D2323542145280
:1052300077625672EAB5CBA5A89589856EF54FE5DC
:105240002CD50DC5E234C324A014810466744764D0
:1052500024540544DBA7FAB79987B8975FE77EF730
:105260001DC73CD7D326F2369106B0165766767620
:10527000154634564CD96DC90EF92FE9C899E989FC
:105280008AB9ABA94458654806782768C018E10870
:105290008238A3287DCB5CDB3FEB1EFBF98BD89BD0
:1052A000BBAB9ABB754A545A376A167AF10AD01AC0
:1052B000B32A923A2EFD0FED6CDD4DCDAABD8BAD1C
:1052C000E89DC98D267C076C645C454CA23C832C10
:1052D000E01CC10C1FEF3EFF5DCF7CDF9BAFBABF70
:1052E000D98FF89F176E367E554E745E932EB23E60
:1052F000D10EF01EEB3C904D53444F53352E3000F1
:10530000020201000110000004F80C00010001007D
:105310000000000000000000000029EFBEADDE41EB
:10532000544F4C20465072696E74464154313220BD
:1053300020200000000000000010000000200000FD
:10534000003000000040000000500000006000003D
:1053500000700000008000000090000000A000002D
:1053600000B0000000C0000000D0000000E000001D
:1053700000F00000000001000080010000000200B9
:105380000080020000000300008003000000040011
:1053900000800400000005000080050000000600F9
:1053A000008006000000070000800700FF0F0000DB
:1053B000FF1F0000FF2F0000FF3F0000FF4F000015
:1053C000FF5F0000FF6F0000FF7F0000FF8F000005
:1053D000FF9F0000FFAF0000FFBF0000FFCF0000F5
:1053E000FFDF0000FFEF0000FFFF0000FF7F010074
:1053F000FFFF0100FF7F0200FFFF0200FF7F0300AD
:10540000FFFF0300FF7F0400FFFF0400FF7F050094
:10541000FFFF0500FF7F0600FFFF0600FF7F07007C
:10542000FFFF0700120110010000004051C20313EA
:105430000001042048010902200001010080320916
:1054400004000002080650620705820240000007BF
:1054500005020240000000040309041C034100543B
:10546000004F004C002000200020002000200020E1
:105470000020002000200028034600500072006930
:10548000006E007400200046006C0061007300682C
:105490000020002000200020002000200020001A12
:1054A000034600690072006D0077006100720065BC
:1054B0000030003000300030000E034D0065006DFC
:1054C000006F007200790000813C000000000000C5
:1054D000B53D0000000000000000000000000000DA
:1054E00000000000000000000000000000000000BC
:1054F00000000000000000000000000000000000AC
:105500000000000000000000F5020000F5020000AD
:10551000B9070000DD070000B9070000DD07000043
:10552000DD070000DD07000095070000F502000020
:10553000F5020000B9070000DD070000B907000010
:10554000DD070000DD070000DD0700009507000013
:10555000F1250000E92500001123000011220000C0
:105560004D270000292B0000452E00009D2E000035
:1055700035240000DD140000FD03000005130000C9
:10558000112200004D2700009D1700000936000081
:10559000A118000035140000433200003D32000025
:1055A00011230000112200004D27000049320000A5
:1055B00009360000613600003524000000000000BC
:1055C00000000000000000000000000000000000DB
:1055D00000000000000000000000000000000000CB
:1055E000005600000000001024010000A445000047
:1055F0002457000024010010FC6F0000B445000097
:10560000000000000000000000000000000000009A
:1056100000000041544F4C20465072696E742800BF
:10562000000000000000000000D4284B3D000000F6
:10563000000000000000000000000000000000006A
:10564000000000000000000000000000000000005A
:10565000000000000000000000000000000000004A
:10566000000000000000000000000000000000003A
:105670000000000013000010000000000000000007
:10568000000000000000000000000000000000001A
:10569000000000000000000000000000000000000A
:1056A00000000000000000000000000000000000FA
:1056B00000000000000000000000000000000000EA
:1056C00000000000000000000000000000000000DA
:1056D000000000000000000000093D000000000084
:1056E00000000000000000000000000000000000BA
:1056F00000000000000000000000000000000000AA
:105700000000000000000000000000000000000099
:105710000000000000000000000000000000000089
:1057200000000000D7EA253997D5BCBD10F9AAD4EE
:105730001AE1A9248DFBD5F1F38BCC0F093F3F1E55
:105740008ABC126E0B279AC823272B9258DCDC9A4E
:1057500034832740D597D0F4847ACF4A575740DD19
:1057600075472F21C51E79AC1F9DCA4AB1B77FF579
:105770005A492D02B7080BD534696DA41F11F74F94
:105780008D3D535FA9E39DE69774B635D588E5DF77
:105790000D05201B80F794FD796269BD2AD8282366
:1057A000670DF5BAE39D67981B1E224C87B6C19121
:1057B00050F4BC491FDB342E33085BBD86A03A147D
:1057C00016CCA713D6D5A26539C2A9AA9822FDD6B0
:1057D000859D070722958B3FD78F37BCAB18BE6AD4
:1057E000668E2D8A7DDCA1D960403365593CA2D1FB
:1057F000032729F9083DED09CD21858AF3BF8C35B2
:10580000D5A02E3DBF08AB7ADB6614ECA2109F68D2
:1058100081E8937D86A7A2D880369E5367A137F191
:10582000AD4FF73B7E0480061A36DA51A9668F9A8F
:1058300033F584C119B6B6039FDD1336D61700F7CA
:10584000631E1765A978C5B4CEA8C5BBF14C418EBF
:10585000768A57758D9027795BA7394D12C0B6CCE3
:105860005103CD87BA4BD895C7C83011A927452415
:1058700071A84982A0F9DC20E1DF1E5C32D23741F9
:10588000784913443DE8AF6795E438638817EF1A09
:10589000AE6942EEA0B31E0DDE836C3858544A093F
:1058A00041EA18676B295001CC1384528B02B35321
:1058B000C8A31FF50B8F73C2B9EB45013EA1EF16CC
:1058C0003D10AFD5CB499304FD5807DDBFC217F497
:1058D000736FD0CD255514DB9590BACCA081850D82
:1058E000F60488F720D1B42A9307BC9813467503B1
:1058F000B966FC3037DBE7FE198D35D8881D664761
:10590000AD135CD60F2C3F1E69B29B41E5BDDCFE9A
:10591000CC23E0797094E0A8A31319D0606877399C
:10592000DE8B448C975B3E5B6C4D8FCCBC4598AF57
:10593000534AFC41CDD76C2CC7ADA61C769DE4EB39
:10594000A0A7B394C08E3630946C912A105B0631B8
:105950007AAC0D16249B5FEFEA9827B55F803EE690
:10596000300687115FA1D343FEAE57B2A5D0D9D37D
:105970002235C70C5730D9DE434CEF869D5FAB2CE8
:10598000514DA77D9A30281C0B03E7A3DB2C6F1A1F
:10599000C9673BA7EAAE489B47C4BFE0139E3D5191
:1059A00073035F5D29D778B62181865F20DABF62F5
:1059B000EAE3B5F9DDF6292DFF7DBE7328F2D19A11
:1059C000C603C91DC5A57AD7D747BA22C44BEE294D
:1059D0001184318CCE1B3D5FE3E70997358BF6AD23
:1059E0002896AB6B53759102F0ABA079A73E598214
:1059F000CE6D48197345AB091BA6AA7F9E8F98B63A
:105A00005CE5A9796F6E729EEBBE7CED35A23870B5
:105A1000C3A365B68C05D12667C646F5FB5C3A7B09
:105A20003D7F70D7CAAD13438EF882A3E903E0949B
:105A3000AB46AD172AFEFFB57E552DC67850F13E18
:105A400006CE0EA6A862CC85F9385B38B10E35F4C7
:105A50003CC6A27FB56380FA5FF684AB6E747A8928
:105A600046735B7CF1BA3E539EE1147AF6970E5C66
:105A70004BA502D689D2ED69A8AA8A453D6398262E
:105A80003F0D9743D81BD88A0992B68C3015D24B5C
:105A90007369E243D23250121FAFCFDD27C0FD142D
:105AA0001F94B2B729BEBC8B4D2A12160195070D63
:105AB000D6E086CD740C67AA61EC1052B59D2DFD21
:105AC00079CADC07CA6D9441F3708A3C2B2206A484
:105AD00035DE5347B34D528927917DEE02DAB4A8E3
:105AE00059A36399892160342EAA5FCB77FE466C57
:105AF0009BB7471936E352EFFE84795D351041D4E8
:105B0000314AEBDA0F14F9914338331C24199FDB27
:105B1000EE444F7EA89DE0BE00002163AB1A0FF655
:105B2000603DA5E34C0E41EAADA1655D2D7264FFB9
:105B30005E40DF6292216AF8F22A4556702D595D67
:105B4000D94AB0ED5A3B8C5040CD9DA78F632FE2D0
:105B500045DB3F36E9350881519C6392B836C8066B
:105B600099668BC2AF54DB58AB291FA57D3BF3E090
:105B7000FB16DD73D3829BF8FE0E83FCEFDF57EA42
:105B800058B9B4722D8789226C7FD93FCEE3A7AC78
:105B9000BC058ECDB66794A48950E8D87A11302818
:105BA000C3B68B25936091935F2718F72CC2F6F646
:105BB000EAB8508B0271D4096E5267B16140CBBA1A
:105BC000ABAD752169BA0FFC8BF51EA91D17D60D5B
:105BD000508D0AD9AE3538A06A91BDA9B674E815C2
:105BE000BD714724A1083E5E7AFDDE5B0D52FC8448
:105BF00048B9C3E176FF84D23F1A2387F6D1EA8CF5
:105C00003E7D8614A467021C6779AD7FA93FA4730B
:105C10008BB9AE14B7B0E855C9EB41BAA4C6DC6283
:105C2000E198D6A6667881E03887333A87309D9927
:105C3000FB82FB920838B0075DE094C48B5609499B
:105C4000E41ABAC75C5C82C9814C1B9379C9A43F32
:105C50003CCBCD64FEDD0AA4505ED4137C27E68ED7
:105C6000A8B7198731A798DFEFA87F80A7C7FF479C
:105C700049A719C343C2DFCA972F591AF41D647A82
:105C800029007C8F042E6C06AD121729EFB9106124
:105C9000B11F20B86798F7D1088A8B860198770ED4
:105CA000F2835DAEA20F566730B1C35D06B11E929E
:105CB000457875A52ADDE1004B43E20AB748C102E9
:105CC00082CD87BA7636B7D2EA993DFD5DFDB00147
:105CD000438FED80D3452E8D326DE038AF8256DD97
:105CE0002079465F2B81F152E3A61F1397D110CB89
:105CF000C1024F27FE2A15B39A78DA64A6F8BA5C77
:105D0000940578DA6C8175CC5807EE9315969E4A07
:105D100022F9ACEE655F7B30BE811E04325C6D3CC7
:105D200046CFBBDF1FB566AE2629CDA13581B109AF
:105D3000FDABE7E38A7DDBEC9C66592CEB4D6FE70E
:105D4000B58B5092B4ACD964906BC876ACF78097A1
:105D500093F0DE1AD7DEF85B1292EE107BC0697109
:105D600016423C19CE3A8F8091FBD0152F0942651F
:105D7000BF70CB06D479FC2C1922BCC9A28390FE3B
:105D8000B21B6430DBE1574425E7B135D3AD9C51FC
:105D9000462E28DD66A34C83D8D03E4144CDFAB5CB
:105DA0002F8278A069051BEF32D9464B16E5467B5A
:105DB000A0C6CC24A33B8F071BFF461761E31EEF51
:105DC0007C57D1027814F6CE85ADBE61ACB3D363F7
:105DD00028BF9864AAC9D99D114925386A3315038B
:105DE0001BBD001587509125E5516F4E8B39411A27
:105DF000B67E38069A4BBB280828E3DD00A312AC18
:105E00003FB0E6172C335A5DEC5A09CEF5E41B6A15
:105E1000758EAE9986C9C5EF2564A55C58C779C74C
:105E2000613723660ED9DFB1AA1C2A44A36CE84867
:105E3000ACFB8B1492B8A34078EF67D5EDC04797C1
:105E4000A57FAE47F99FA930E7E6DB5B415494F5A7
:105E50009DDF0B204870F1DE17400A4A8A71B57D3C
:105E60006BA109286BCBCE404540C0F9A50676F260
:105E7000F1AC13DBCCFD0B07930C4E6129C5393116
:105E80007E4C19A32A3650E3BDD59DF542B43B4A5A
:105E9000281A104908B91C56057EA9331FF8E617C1
:105EA00069D89A9603ACF676887AA4937112CE4894
:105EB000234E1FC4ACA60409D89DE2F1F7C7EC99A4
:105EC000E27CD8C2BB6D7E4EDBAC81D4CF20647641
:105ED000C9B7D232983146E7E973262159EC8DC211
:105EE000B2C977CA777C63A65DC8CFACBC0B4DCE78
:105EF000C8291E9A3C36281D4FB957EBCB8C00FFA2
:105F0000D7AD2E6CDEEAB1F0723334F3922E8F05EA
:105F100005CE915482100FAEF7CB52B6195E946F36
:105F200021CDC1FCA93A568A61FB995AD1FE71C3B1
:105F3000B21D6A6A9C44EB34AF5519B983E3509A99
:105F40009F14FFB91CE9403AA2DA2FF2C2F3AE4225
:105F500097C59BD426C07894E00FC692BB2BC31282
:105F6000DC357FCF919B059391D11A0A5A12BAEA78
:105F7000F7803F66214962BA52907DD65728C544C2
:105F8000F1E7DE59FF29FE7784F4AEC677FC95F37E
:105F9000E05168BEA00EF2CA1DE6722DF906127617
:105FA00043CC1455D388249AA6B248F4D0FF69EFA5
:105FB0001F1D29469CD3DE1DC972333225920BF476
:105FC00048683474BDCD8F5EB6CC8D86BE56826077
:105FD0007275D3C90D64EEE872FDBF5112980A685C
:105FE000AA2CEED422749DD1C7BD9E67C0D198570C
:105FF0004CEA2DE494C3B9C5AA8639A879BAE1A5BB
:00000001FF
